:020000040000FA
:1000000007309F0083169F011E308500F030860068
:1000100081138312EF30A40086000430A000A40CEA
:1000200024088600382006080F38A100A109031D06
:100030001C28A00B0F280A28831600308600831284
:10004000A40924080F39A4002108F039A4042408C5
:1000500086001130A100A103210840202402031DC5
:100060002B282108860010302107402086003728E1
:10007000FA30A300A200A20B3B28A30B3A280800E9
:1000800082071134123414341834213422342434C5
:100090002834413442344434483481348234843402
:1000A00088343034313432343334343435343634C3
:1000B00037343834393441344234433444344534A9
:0200C0004634C4
:02400E00293F48
:00000001FF
